Subject: [babel] Babel over DTLS

From: Juliusz Chroboczek <[email-masked]>
Date: Sun, 11 Mar 2018 17:38:37 +0100

17:34:25.800782 IP6 fe80::a6b6:7003:d50:6868.6696 > ff02::1:6.6696: babel 2 (8) hello
17:34:25.801038 IP6 fe80::a6b6:7003:d50:6868.6696 > fe80::d17a:7827:dae0:58f1.6696: babel invalid header
17:34:25.801075 IP6 fe80::a6b6:7003:d50:6868.6696 > ff02::1:6.6696: babel 2 (24) hello ihu
17:34:25.803681 IP6 fe80::d17a:7827:dae0:58f1.6696 > ff02::1:6.6696: babel 2 (24) hello ihu
17:34:25.803944 IP6 fe80::a6b6:7003:d50:6868.6696 > ff02::1:6.6696: babel 2 (24) hello ihu
17:34:25.804240 IP6 fe80::d17a:7827:dae0:58f1.6696 > fe80::a6b6:7003:d50:6868.6696: babel invalid header
17:34:25.804298 IP6 fe80::d17a:7827:dae0:58f1.6696 > ff02::1:6.6696: babel 2 (40) hello ihu ihu
17:34:25.804518 IP6 fe80::a6b6:7003:d50:6868.6696 > fe80::d17a:7827:dae0:58f1.6696: babel invalid header